:020000040009F1
:280000000108006999994204204EB1FD0400FFFFFFFF4006009376A0027020020A002800090000000000000014
:FB002800411A0042726F6164636F6D20426C7565746F6F74682044657669636500980100035C0100017206000300000800019304002400000068040012000C006A3600030111000000B0000000A0000000431008045310080480000000900000006310080473100804C1000000D000000022000000320000007C04000100000209080068000F00030000006F210002331F05CF000000AA147F8C00AA00800A9200000000140000000000006C584E6CA1040000000080690200E3065D0C000A64E6B000008898425A33435F09003C280100040004F70C0A6F0098160800C600F3025D0066033000C900E10268005C033600C300E2026A0053033C00C200E102D4
:FB0123006C004E034100C500D60272004A034300C300CE02790042034800C500C00283003A034E00C800BF0282003B034E00C900BC028400370352000808070707070707060606060505050502C0500194FC0E00FFFF00005E02000030FC0E00FFFF0F006304000000FD0E00FFFF0F006602000088FC0E00FFFF0000000200002CFC0E00FFFF00004904000070FC0E00FFFF00000B09000074FC0E00FFFF00002E010000D8FF0E00FFFF000062190000D0FC0E00FFFF000020C90000C8FC0E00FFFF000038850000DCFC0E00FFFF00001CC80000CCFD0E00FFFF0000048000005CFC0E00FFFF00000200000020FC0E00FFFF000019210000E0FC0E00008000FC
:FB021E000000000000C0FC0E00FFFF000022000000948F0800FFFFFFFF00120012988F0800FFFF0000001200009C8F080000FFFFFF0004040478000F00FF0000FF0500000030010F00FF000000050000008C000F0000F0FF0F0000800034010F000F000000070000001C010F000000FF000000250074000F00000000FF000000300C010F00000000FF00000030B0010800FF0000000500000068000F00FFFF000003000000D07B0001040A08FC0E00FFFF00002E3600000CFC0E00FFFF00002CAE000010FC0E00FFFF00002AAC000014FC0E00FFFF0000A222000018FC0E00FFFF00001D2000001CFC0E00FFFF00000D15000020FC0E00FFFF0000858D00000B
:FB03190024FC0E00FFFF00008311000028FC0E00FFFF00000001000098FF0E00FFFF00003E410000C3160012651428783F0444306070047180764A3108290B7E07CF090010000F6EF0B009F060D10900010403036B1438206B1A2400FF00080804120010FC0EF80CF40AF008EC06E80404120010FC0EF80CF40AF008EC06E8040301000182D600040602020A233C5A6E7D80008000800080008000800080008000800080008000800014FF38840AFF610000000000000000000000000014FF38820AFF610000000000000000000000000014FF38000AFF610000000000000000000000000014FF38050AFF610000000000000000000000000014FF380B0AFF6B
:FB041400610000000000000000000000000014FF380D0AFF610000000000000000000000000040FFFF68027B0000000040FFFF68027B0000000040FFFF68027B0000000040FFFF68027B0000000040FFFF69027B0000000040FFFF69027B0000000082D600FF0602020A233C5A6E7D80008000800080008000800080008000800080008000800014FF28840AFF200000000000000000000000000014FF28820AFF430000000000000000000000000014FF28000AFF660000000000000000000000000014FF28050AFF660000000000000000000000000014FF280B0AFF430000000000000000000000000014FF280D0AFF20000000000000000000000000009A
:FB050F0041000000007B0000000041000000007B0000000041000000007B0000000041000000007B0000000041000000007B0000000041000000007B000000008612000413004008000040130001000180FF000112C15E0044041422A244041422A23B04B104B204B304B404B504B604B704B804B904BA04BB04BC04BD04BE04BF04C004C104C204C304C404C504C604C704C804C904CA04CB04CC04CD04CE04CF04D004D104D204D304D404D504D604D704D8280C000B0400222A09000B04001C2B09000B0400462D0900081D00005018010081F008FD0E006432090030B4201CFFF7CCFF30BC7EF7FEFA08190001086501007CF0B3FE0A0072320900FFF7F6
:FB060A00ABFF83F761F9000008250002B0DB010076F01CFD1600EC450900281CFEF74FFE281C5F3000210170391C321D89F7D9FA080F000384E0000030BD00B50000000000000817000488E0000085F0B8F90800FC33090000F002F800BD0000081D0005C46200008DF0C9FB0E005A3A090001B4FFF769FF01BC72F739FC000008150006586600008DF0FCF90600543A0900FFF796FF30BD0B0400FA3B0900081F0007484800008FF060FD10000C430900A56498231D53201C00F002F870F799FA0B0400243C090008150008C08400008BF0E2FE060088420900FFF7A6FF30BD08350009B47702006CF06BFD26008E42090002B421684907002905D06168492C
:FB07050007C90F301C93F70FFC02BC002902D0F06993F784FA93F786FA080F000A24B500000FE0C046000000000000080F000BC44F000010E0C0460000000000000867000C1CF0030055F04AF95800B442090070B5061C0C1C151C002B21D104A8008840281DD105A80088202819D15A2917D8081C15D005F0F0FA002811D1032D0FD02204121408210748002305F0EDFA002806D1221C291C301CAAF74DFF012000E0002070BD18650800080F000D988000005808042B0000000000000817000E680C040053F068FB08003C43090000F002F870BD00000819000F64D4000086F0ECFF0A0040440900281CFEF7A7FE79F722F80813001008D6000086F01FFFFE
:FB08000004004A44090079F7E0F8080F001180DA0000C046C04600000000000008150012245200008FF013F906004E44090000F001F8F0BD0B0400B045090008190013845C02006EF0BDFC0A00024609009B005859EF1891F73EFB0817001464F8000084F0D2FE08000C46090000F002F8F0BD0000081700153CF5000085F0D2F80800E446090000F002F830BD0000082F0016C4F6010075F04CF8200060470900054B30B4054CE57949190C06211630BC19548AF7A9FFC046903408008C03080008170017487C02006CF09AFD08008047090000F002F870BD0000082B0018D4BA000088F090FE1C00F84709000AB4201C311C00F009F80ABC012803D0042BB5
:FB08FB0001D177F764F977F765F908250019E4A203005AF0A3FA16002E480900002803D000F007F8002802D10120A5F77EFDA5F754FD0817001AC06A02006DF0DCFE08007C48090000F002F830BD00000823001BC47202006DF07AFB1400BC49090008B4301C0122012300F004F808BC92F77FFC00000817001C2C6A01007EF0A4F80800784B0900FFF7DDFF00BD00000815001D98AE020069F086FE0600A84B090000F00AF870BD0817001E0C13010083F04FFC0800AE4B090000F035F87CF7AEFB0819001FFCBE020068F05BFE0A00B64B0900281C00F03BF897F7A3F9087B00200C7702006DF09CFA6C00484C0900F0B5061C0F1C93300078002803D00BC1
:FB09F600795B08072B24D17DF7F4FE041C0C301422391D051CBFF78AFE7268002A03D0291C301CC6F719FE3368E3770023A37709490868002804D00368236004600C6001E00C6024600121890403480022B8F7ECFDF0BDC046ECC40800FC440800080F0021587B02006DF0ACF80000B44C090008230022B47102006DF0A0FD1400F84C090002D0E86992F75CFA281C211C00F002F892F76EFA081F00239C6E02006DF04AFF1000344D09000FB4201C00F004F80FBC92F7B1F80000081F002408F0000085F0A8FE10005C4D09000FB4201C00F004F80FBC7AF763F90000081B0025B86A01007EF072F90C00A04D09002961EC607AF732FB81F789FE08210026C7
:FB0AF100F0D0020067F084FE1200FC4D09000870684610B4FFF7EAFF10BC6B4698F773F9080F002728EA0000F0BD00B5000000000000081500282CEA000086F0EFF906000E4E0900FFF7CDFF00BD58010037081B0029DC8302006CF038FD0C00504E090093F73FFDFFF7DEFF93F7C2FA081D002AD83C010082F0B9F80E004E5E090001D17DF761FF281CFFF7EFFFF0BD0817002BBC6504004FF0CEFD08005C610900FFF7ADFE01B0F0BD0815002C746604004FF076FD060064610900FFF7D7FEF0BD081D002D105D040050F02BFA0E006A6109000FB400F00EF80FBC2068AFF7D0FD0819002E785F040050F0FEF80A00786109000FB400F00FF80FBC10BD08B6
:FB0BEC0019002F985F040050F0F3F80A008261090000F021F8AFF723FF000008150030D87304004FF032F906004066090000F01FF830BD081500318C7E04004EF0DBFB06004666090000F045F870BD08150032507F04004EF07CFB06004C66090000F0BDF830BD08170033A07F04004EF057FB08005266090000F0EAF802B010BD08150034788104004EF06FFA06005A66090000F050F910BD08150035188004004EF022FB06006066090000F06AF900BD08150036FC7E04004EF0B3FB06006666090000F06FF8F0BD08150037B08704004EF0F8F80600A469090000F004F830BD08150038348904004EF039F80600AA69090000F0CFF870BD087F0139A444E2
:FB0CE700000092F0DCFC7001606E090000B528490B6826490B6024490B6822490B601E490B682D490B60434B43490B6034490B680120C00303430B6040490B78002B04D02F490B68400303430B602D4A13685B085B0013603A4B3B4A1360B2F754FAB2F77DFEB3F7CCF9B3F772FB0D21364802F023FD364A9068002803D09AF77DFBB2F719F92448244A11684160244A60E0C046C0B00800FFF2011ABCA30900848FB002D08B0E00A0800E00C0A30900148B0E00C4A309006CE50500C8A309008C150800476D0900776D0900516E0900CD6D0900396E09005C000F0094830E00FF00FFFF608B0E0040230001E08A0E00E02C0800A4860E0088B208000500001C
:FB0DE20080850000801C800E0014800E00848F080004830E00108B0E00C8FC0E00C42C0800CC2C0800D02C0800C82C0800D42C0800D4FF0E00BC8B0E00AD020000CC8B0E001CCD080010325476D48B0E00009D0800ECCC080011684161054A11688160054A13680360044A1368044A136000BDC046D02C0800C82C0800D42C0800D4FF0E000861003A0044000092F026FC5200506C090010B5A448002383700423437001230370A14BA2480360A24BA24C2360A24C2368A24C2360A24C2368A24C23602C22A249A248BDF77FFEA148A14C2060A149C160A1494162A1490161A14B8361A14BC36110BD080F003BD0B80400A5F809E00000000000000817003C9B
:FB0EDD0020BA04004BF08CFE08003C770900FFF7D4FF30BD00000817003D3069040051F010F8080054790900FFF7C4FFAFF708F80819003E545D040051F002FE0A005C790900B5F780FAFFF7B2FF30BD0819003FE0A504004DF0C1F90A006679090000F003F803B0F0BD000008170040E88204004FF090FB08000C7A090000F002F830BD000008170041B0B104004CF0AAFC0800087B090000F002F830BD0000082B0042DCC004004BF098FD1C00107C0900FF233D3343430448C0189F300078002800D101207047C046349D0800081B004394AC04004CF0D4FF0C00407C0900201C00F003F8B3F728F80000081B0044ACAC04004DF014F80C00D87C0900207A
:FB0FD8001C00F003F8B2F7E8FF0000082300453CC104004BF076FD14002C7C090029187F231B02FF339D4200D35D1EFF23B4F780FA08170046981B030066F016F90800C87D0900FFF7D2FF30BD0000081F004718AC04004DF016F91000487E090003D1FFF7C1FFB2F7E6FEB2F7E5FE0000080F00481C730400C046C04600000000000008150049807A040050F0B8FA0600F47F0900FFF7B8FF10BD0815004A988204004FF0AFFE0600FA7F0900FFF7C9FF30BD0817004B6CA804004DF07CFC080068810900FFF74AFFF0BD00000815004C94A304004EF0B5F9060002870900FFF7E5FF10BD080F004D0CA3040000F01DF80000000000000823004E489400001E
:FB10D3008FF05EF9140008870900012B02D10020287001E070F7A5FE626870F7E1FE081F004FA4CC04004BF03AFD10001C8709002878B3F742FA201C00F002F830BD0000080F0050C4A904005E4A2068000000000000080F0051A4630400FE23F533000000000000081F0052D472000091F034FA100040870900301C049900F004F8009988426EF7C4FD08170053989704004FF000F808009C870900FFF705FEF0BD000008150054D09901007FF0A4F906001C8D0900FFF7B2FF00BD0815005568E901007AF0DBF90600228D0900FFF7C2FF00BD08230056A4E901007AF0C0F91400288D09000FB4301CFFF7C6FF0FBC0A22311C85F737FE0000081700577037
:FB11CE00EF000089F020FF0800B48D0900FFF7C2FF76F7E0F8081D0058645F040052F02AFF0E00BC8D0900607D01386075FFF7C7FFADF7D0F808170059E85E040052F06FFF0800CA8D090076F7CCF8ADF795F80819005A14FF000088F05DFF0A00D28D0900FFF7DEFF77F7A2F80000080F005B6C5F040000B5001C0000000000000815005C705F040052F062FF0600388E0900FFF7EBFF00BD0829005DD07E000090F0B5FF1A003E8E090009D5281C112806D0082804D0002089F738F86DF74CFA30BD00000817005EEC6B040052F076F90800DC8E0900FFF7BCFF10BD00000877005F7461030062F070FF68005890090010B500248DF730F8012803D309D077
:FB12C900022820D102E09FF77AFC01E0A4F7E2FF041C18E00D490B78002B14D00C4A106803680B4A13600B4A1378002B0BD08B784978002B03D04B00FF21013101E04B00802199400160201C10BD481B0800E40A0800AC5808003A010800080F00607C640200131C036000000000000008570061B462020072F004FF4800C090090000B50D490868002804D003280FD0052811D104E009480378002B0CD007E0084B1868012200219AF74CFB9CF71EFF05490B680120186000BDB0C80800D1CA0800F40A0800E40A0800081B0062C0B903005DF0A2FB0C0008910900211C00F00BF8061CA2F75AFC081F0063B49D03005FF0AEF910001491090002B400F015CB
:FB13C400F802BC0C68E306A0F74AFE081900647847000094F07EFE0A0078940900381CF9F77BFC6BF77EF908190065AC47000094F069FE0A0082940900281CF9F794FC6BF797F9081B00663CDB00008BF0A6FC0C008C94090081B000F003F874F7B8FB000008270067405B010083F01AFB180078910900002E02D00020E05504E0E35D002B01D0013BE3557CF7F1FC081B006850A704004DF000FC0C00547F0900381CFFF788F902B0B2F7FAFB0817006958A704004DF002FC0800607F0900FFF7A9F9B2F707FC0821006AB03C010085F0AEFC12001096090001B4301C00F010F801BC75F753FD7AF749FB081D006B5CB503005EF061F80E002296090001B497
:FB14BF0000F00FF820BC6B01A1F798FF0817006CA8A003005FF0C2FA08003096090000F015F8A0F754FD082B006DCCB203005EF0DEF91C008C9609001378002B07D103B400F008F8012803BC01D1A1F718FEA1F722FE0000081B006E74B403005EF024F90C00C096090000232B7500F02CF8A1F7D6FE081D006F1C69020072F0D6FE0E00CC96090003D100F027F8A3F789F88DF724F90827007030BB03005DF0D3FD1800DA960900012D03D1002E01D100F05BF8A068A2F7A4FF0021A2F722FA082700710862020073F073FA1800F2960900201C08B4019900F01BF808BC9C4201D08CF783FD8CF78DFD082500729CBC03005DF035FD16000A9709001B070570
:8015BA00D400F049F8002801D1A2F7C3FAA2F7EEFA00000A05002DCB080001081B007330AB03005EF042FE0C00B897090005B400F003F805BCA1F7B8F90817007498C803005CF0A6FF0800E897090000F002F8A3F77CF8081B00754CD303005CF088FA0C0060980900800D00F00AF8A3F774FD00005B0900FD0344042804080803FE000040
:FB28E000F0B5554C554B56480360564B56480360564B57480360FF232D335648038000F0BDFC00F072FA00F025FC00235248037000F080FB00F092FB04F093FC06F0E2FA4E4A151CE4354E4B2B604E4E3368022633434C4E33604C48036880218B43036000234A4E33704A490B1C2333494E3360494B4A4E33604A4B4A4E33600B1C1233494E3360494B4A4E33604A484A4B4B4E3360031C0E334A4E33601223494E33700B1C1133484E3360484B494E3360494B494E3360494E3160494B4A4E33604A4E33684A4E33604A4B4A4E33604A4B6B674A4B061C071DC8C40E36494FC8C4991C0E30061CC2C4474BD3620023464E336005F06EFE454B6B65E420A0BE
:4729DB00F743FC002343490B6043490B704348E86243490B6843490B6002F0CEF8002342490B70A02341490B70002341490B703948036801210B43036002F024FD02F064FEF0BC08BC1847CD
:FA2A220000B53A483B4908603B480B49C86400F098F900BDC046E09A0900C9320900BCC80800DD320900F0C40800C53209000CC5080080020800DDA40900A0190800253409006C010F0040150800FD0708001E4500001C9B090020C90000209B09001CC80000249B0900289B0900388500002C9B09005E04000044050000881308008C13080090130800781308000EC90000801308000AC800007C130800841308002685000074130800D8FF0E00309B090062160000349B0900D93909004205000062190000597E0900189B090049470900389B090064A40900D18B090028FC0E00E803080065A4090054150800089B0900E128090090000800754509008A
:50992C0023000000712B0900240000006D2B090025000000752B090028000000ED4A09002E000000954D090035000000AD2B090088000000ED2B09008D000000112C0900910000006F93090092000000000000004F
:502B1C0070B500200F49104B4B6114E06B099C00EB06DB0E01259D400B592B430B5143004C69C50052195268012632432725AD03AA1A1A530130054AC3009D58922DE5D370BDC0464C1B080050A409002C990900EF
:042B6C00002070478E
:042B7000002070478A
:382B740000B5002812D0AC231A581204D20E0F290ED1012A03D0042A01D0062A02D178F7FFFF03E0002A01D0032A01D1012000E0002008BC184700008E
:042BAC00002070474E
:242BEC008105890D030AFC201840FC2803D1F72901D1034800E000207047C04664A40900B12B090040
:282C100004280AD106480378002B06D0054803785B065B0E0370012000E000207047C04664A4090039C30800D3
:3C2BB00010B5037814490B700620ABF72DFE041E10D00E230370042343700023437101238370F723C370FC230371ABF747FE201CABF71EFE012010BC08BC18479F
:FB2C380070B5051C0E1C80780002697808438205920D030AFC2018400C280BD1032A72D102F008FC02F04CFD311C281C06F0C9FA012069E00124FC285ED1342A35D0C62A5ED319D0C82A1CD320D0CB2A23D9E62A0DD0E92A24D0FF20313082423DD0013082423FD0FF207930824249D13FE0311C281C04F091F944E0311C281C06F0D7FAD6E7311C281C06F00FFBD1E7311C281C06F04AFBCCE7311C281C98F7ADFDC7E7311C281C03F0BEF8C2E71B490869C00126D51A4A106920431061101C117D8B0706D5FD231940017500207FF752F817E0002103207EF7AFFF12E0311C281C06F061F8A5E7311C281C06F06DF8A0E7311C281C02F097F804E020280436
:132D3300D0042802D10024201C00E0002070BC08BC18470F
:1A2D46000448044908607047C04654200800CC2F0800392C090018C90800DF
:042D60000020704798
:102D64000148024988607047612D0900201A080053
:082DEA0077487749C860704783
:FB2DF200F0B583B0041C012906D164300023C372251C9435AB73EB73714803689B079B0F032B02D073F769FAC8E00023A381E07B484000D1B6E072F704FD002803D1684803691B0101D5012100E00021271C64373E1CFB6880208343C8010343F3600C36614A1078431006D0C3071B0E316880208143194331605A4803691B0102D4381C96F7E1F9BB69002B02D03B681B063BD4338868460380E37B012B0DD0251C94356B7B002B10D02B88042B0DD3EB7C022B0AD3AB7D002B07D1A72303201855009B78208343002106E00121E974009B78208343082003431F20800283438802034300931B041B0C404A1360012030723C4A13691B0152D40098400601E2
:FB2EED000F00231A1C012096F7C1FB45E0E07B002802D1A72301221A55012804D1E37C042B01D074F7B4FCF37A002B06D00023F372336801204002434033600121B172251C9435A97328480369DB0002D5201C89F7C4FD338826490B60B0884860381C72F7E4FC30684006030F2248C05C3072431EA381E37B002B0FD10121387F81401D4A1068084008D1E37C042B05D01B480378AB751A480378EB75134803691B010FD5201C96F71AFF0BE0271C64373B727B7272F772FC636C002B02D05A231B5BA38103B0F0BC08BC1847C04609C108003C9B0900000408004C9B0900F32D090000020800188B0E0054200800DCC80800CC8A0E009EBB0500B401080072
:082FE800F5010800F6010800E4
:022DE800704732
:2830140000B52C2204490548C1F7B2FC034804494161044B186000BD0CBD0500CC9B0900F12F0900E40208007E
:242FF00030B50D1C041C77F7B5FE6B075B0F012B05D1E37B002B02D1A07B9EF7F4FD30BC08BC184784
:18303C0010B53F4C3F4B1C602C223F49201CC1F79BFC3E48606210BDB0
:FB305400F0B5041C051C876A28353B4B42331878002866D1201C012174F70FFA061E4BDD022804DB201C79F789FA002859D1618C8B1F9E4223DA304A13689C420BD0391CAB310878013800D30870731C5910201C79F716F830E0731C5810E37B002B05D07B6C002B02D06B7F002B25D02F89B84222D36A89002A06D1A389002B03D1201C73F71DFE18E0BA4200DA3A1C904201D90C2310E04B23A27C1B5D9A420CD102280AD36B7F002B05D014480378994201D9282300E03823A374211C4D31087800280FD00238087000060BD1E37B012B02D0237D0C2B05D0321C201C0523022179F772F9F0BC08BC1847F89B09000003080074BD0500553009006C2108B5
:05314F0000F40208007D
:1831540000B52C2216491748C1F712FC1548164B18601649016100BD28
:28316C0030B50D1C041C7AF75AF8022D09D16B23185D002805D0201C89F743FB201C89F77BFB30BC08BC184706
:0831C40000B57EF790FA00BD92
:5432040010B5011C2831041C7BF7C1FC002819D0F8210B585B0706D4C3699B0219D40E4A13681B0402D5FFF7CFFF12E0E3698B4310200343E36199230B201855201C83F74CF906E05023054988881853201C94F7C1FB10BD59
:3831CC0010B5041C031C9A3313201870E3691B06DB0E0A2B03D10A21201C7DF76AFA201C83F73FFA201C83F76AFB201C83F756FA20687BF7B2FE10BD1A
:0C3258007047C0468C070800D420080016
:14327C0000B52C220B490C48C1F77EFB0A4B0B48036000BD9A
:343290000A49CB6ADB0007D5094AD3885B00418C8B4201DC012100E000215A3001707047B0CB0500509C0900F40308005420080094200800CA
:0432C400002070472F
:1432C800087B4008072801D10148886000207047E14A0900EA
:3C33C0000C480D4908607047F4440800284508009CBE0500FFFBFFFFFC440800FFFF7FFFC04F080065A40900E44E08001C450800FF7FFFFFDD320900F0C408001C
:E432DC0030B5041C002969D0012958D1400520D426E0364D291C3648B9F7A3FF2988281C262902D104F017FB13E0042902D17EF7EEF90EE00F2902D105F046FA09E0272902D103F0A5F904E089002A4A8958C8F7C4FA2748B9F79DFF0028DAD0264B1C4020020AD57CF7C6FE0121C905234800230122B9F75EFF224B1C4020042ED521490868037920490B7000230371B4F705FF7BF792FE002803D11C48437D002B09D01B487CF7C4FE83F70DF81321162005F0EFFC01E07CF77BFE164B1C400EE002290CD1C00308D510490878012804D10D490B681871B4F7D6FE7DF769FF201C30BC08BC1847E1
:2034040000B5431E04490B6004490B78032B01D1C1F778FF00BDC046E08A0E003808080058
:FB342400F0B587B0061C0491081C00210391A34C2064211C4431009100238B70A0488568002D00D16EE2AB7D002B09D0012203920023AB756361237810208343237006E06069002803D0012E01D972F791FE22691D27FF03002A50D0607A012803D19389002B4AD047E08F4B1B5C002B43D1BB68DB0742D4137D092B3DD204281AD1012E18D196756261237810200343237023683B6085490B687233187802282DD0002382490B608249086882490B6803600B68036022E002280AD1012E08D196756261237810200343237023683B6015E0032803D179498B78022B0FD0062801D0032805D1012E03D1BB689B0600D5C0E1122803D0102801D072F7BBFD6ADF
:FB351F004B985D029000287DD00123DB07334301936B4B6C490868986301236B490B606B490B689B0C9B040B600B6869490868034366490B6001230099CB7066490B6866490B6066490B6866490B60287C1A281DD164490B6864490B6064490B6864490B6064490B6864490B6064490B6864490B6064490B6864490B6064490B6850490B60634908686349086063492DE063490B6855490B6062490B6855490B6061490B6855490B6060490B6855490B605F490B6855490B6019280ED1FF2017302B562A3309DD5B490B683E490B605A49086851490860594908E059490B6839490B60584908684C4908605749086857490860A87B2318042801D3187800E065
:FB361A00205C6F2290431870C2E0A87B225C0F218A433107090F0A43225423180428049802D38107101C01E081071878490E6022904308431870234B464908689863009AD378002B00D1A1E022490B689B0C9B040B600B684049086803431D490B600023D3703D490B681D490B603C490B681D490B603B490B681D490B603A490B6821490B6039490B681B490B6038490B681B490B6037490B681D490B6036490B6809490B6035496BE0642C08006C210800ECBB0500DC02080060000F00AC2C080044020800882B08002CFC0E0060020800E08A0E00B88A0E005C0208006C130800D8FC0E0070130800E0FC0E001C9B0900CCFC0E00249B0900DCFC0E0020A4
:FB3715009B0900D0FC0E002C9B0900C8FC0E00289B0900D4FF0E00F89A0900FC9A090030FC0E00009B0900781308007C130800801308007413080084130800E09A0900E49A0900E89A0900EC9A0900F09A0900F49A0900D8FF0E00B82C080048020800BC2C0800C02C0800C42C0800C82C0800CC2C0800D02C0800D42C0800D82C0800DC2C080008689349086093490B6893490B60002101912868826A281C0021C8F77DF8002810D026231A5C002A0CD08368002B09D00298002804D0802301981843019001E0012200E00022237880208343D0010343237020200499084001D00120C0037F4908600499090704D47D490B68802083430B600499880801214B
:FB3810004140A27880208243C8010243A2702868826A281C0321C8F743F874490B78012B01D078F7E3FF05A9714A13687020034018099EF730F82369002B14D0637A032B11D18AF791FB002806D16A480368032B02D00368062B06D12B7C122B03D101230098837058E005988007800F06D003280ED1069B60490888834209D30398012800D1656172F7FEFB012300994B7043E00820B860A87B786223683B603B1C1833221D03929207920F02D1039909680FE00399891A0391D2000968D140049120218A1A03994968914001B40598014301BC1960BA69331C103B042B0DD2474B1340FF22013282401343BB61102E07D1444908684449086002E04048104C
:27390B0040B8610198002800D07861E5602672002300990B704B70281C8EF745FC012007B0F0BC08BC184752
:5439840010B5254C234B607A185C002802D072F7EFFE15E06069002801D072F7F9FB27490868637A012B01D1254A00E0254A13680360116801600023234A136072F704FE002322490B60E3602361637244340120207010BD6F
:52393200394B3949087A185C39490B68002814D00120800303430B60364A136836480340364A117849020B43354A1360354A1368302083431020184308E0324803400B602C490B682E490B602E4908682F4908607047AE
:7C39D800002803D103480368034803600020704730FC0E00309B0900D8FF0E00648B0E00A4860E00D4C1080024860E001C840E00E4B60800FFF0FFFF9406080064FC0E00ECBB0500642C0800808B0E00B02C0800FFC1FFFF9013080088FC0E00B42C0800FFBFFFFFCCFD0E00AC2C0800400208004402080060000F0018800E002E
:2A3BFA000948044988617047C046C4C408006C2108000C2D0800201A080024860E006602080064020800693A090073
:FB3A680070B582B0061C65480168890602D5022074F7AFFB624C2568A3682360002D26D0002E18D1A0F784F9002814D0C30703D52A68916900290BD1430703D52A68D169002905D1830706D52A68116A002902D0281CC7F7FCFEA0F788F9011C2A685269002A04D0002802D0281CC7F7EDFEA0680026A84218D0002D21D02A681269002A03D0281C0521C7F7DFFEAE8123699D4200D126612B7D092B11D3281C75F778FD281C75F7FDF80AE0002808D06369984205D166613B4800220121B9F7ADFE3A48C16E002904D0A368002B01D1C7F7BFFE72F746FBA06800284BD08681037D092B20D26369984205D166612E4800220121B9F792FEA068A84206D10152
:973B6300684968002902D00523037508E0017D032901D0042905D101684968002901D0C7F798FEA0680223037501680A69002A02D00221C7F78BFEA068807B1D4A136870210B401909884216D169469DF77AFE72F7F0FB002801D0174800E01748028800998907890F04D0032905D1019B934202D33F2301201855A0688EF770F901208EF780F9A66066603C3426716671012002B070BC08BC1847F0
:20431C00A823195C002903D0011C64318B8ECB86011CC36F6431002B01D08B8E0B877047E7
:083C24009E489F498865704726
:643C2C0000B59E4A9007800F01D1116808E0121AC0001368C3402021081A516881401943C90F97480170974A1068002817D0964A0260964A8260964AC2600123954A13700023954A1360954A1360954A1360012902D100F007F802E04068C7F715FE08BC18470000FC
:0C3C900000B500F003F808BC1847000065
:FB3DC000F0B585B0071C0B1C0A1C514D002600960190011C02AC0BC401235B024D490B604A490868030C1B046B602E6053004A481C5A4A498C4211D18023D85D484A835C1B01484818188388002B07D0434C1034837A012B06D1414C203403E0002C01D12C6018E1381C8EF749FB002800D040243D480368002B07D0602C01D1E024ADE0702C0BD1D024A9E00498042801D0022804D12B680120000403432B60302C06D17023D85D002802D02C4C703496E0502C0BD13B6FDB052B6804D50120400403432B608BE029480340FAE7244B30339C4255D101992031C87A002849D1061C79E02D3C0900A0190800C005080030C8080044060800913C0900C13D09D9
:FB3EBB000069400900B805080034C8080038C808003CC80800D005080040C8080048C808004CC808009C800E0010800E00FFBFFFFFFF030000BC820E0010000C0068500800673D0200D405080070010F005C000F0074820E0098A409000C800E00D8050800100100009005080024500800D4C40800FFFFFDFF0128B3D00228B1D003282BD1AEE7984B60339C4213D1039880304278002A01D1161C02E0022A00D10126837E012B00D10226437E012B00D10326330688E78C4B40339C4212D1029B28335879012801D0002800D1061C02990B8D58107F2801DC43062B603306286818432860286820437F4B70339C4203D023097E4AD15C0091302C0BD1702361
:B23FB600DA5D002A07D13A1C2832137D927A99180906090E009100990B0318432860FB7B002B04D06B680122D20313436B60FB7C032B0AD13F2212027B8C5B103F2B01DA9B069A0C6B6813436B60402C28D168490B78002B08D0381C8FF7CFFD03071A0A2B6813432B601BE00122D20402432A60B87B9DF757FC40085F4908605F4A11689DF7EBFB5E4908605E490B68984204D2381C8FF792FD002802D00123554803702B68584803606B68436005B0F0BC08BC1847E5
:D4406800F0B582B00F1C051C0022009201908EF721FA504E002844D034684948017800291AD1A87B9DF725FC4008464A1060464A11689DF7B9FB454A1060454A1368984204D2281C8FF760FD00281BD001233C480370414B1C4015E06B6E1B0612D4012910D1281C8FF750FD00280BD1A87B9DF700FC4108344A11600023314A13700123DB041C432E480378002B03D001988EF78AFE0090314B1C40009803071B0A1C433460042F01D0022F05D13368012109040B43012107E02A480378002B06D0336828490B40002133602548017002B0F0BC08BC1847DD
:B83C9C0010B564238B48037000238B4803608B4803608B4C236000F04FF87C4A9007800F01D1116808E0121AC0001368C3402021081A51688140194301204007014015D080490B68001403430B607F490B687F4803400B6004390B680120800303430B607B4B7C490B6003037B490B60674A9007800F01D1116808E0121AC0001368C3402021081A516881401943C90011D5734C2368002B02D0201CB9F795FB7049201C00231A1CB9F770FB6E480168201CB9F776FB90F7F2F910BD4A
:6C3D540010B56B4C236801242343694C236001239B03684C23604F4A9007800F01D1116808E0121AC0001368C3402021081A516881401943090105D55D480368022003435B4803605C4800218160F421C16020210161E8218161E9214161102141624021C161016205239B04036010BD82
:B041D80030B5041CC37C032B27D1037D0C2B24D11830437B002B20D121490B699C4202D18B68002B13D0418900680B1858010509A07B9DF766FB854201D3281A03E0431B01200007C01A831F1648834205D3201C75F7E6F9201C74F774FE237D022B03D0032B01D0042B07D10F480379002B16D0201C72F7BDFC12E00C480369002B02D0201C71F752FF06494123585C012804D0002804D10B689C4201D174F7E0F930BD6C210800FBFFFF07A42C0800642C080000
:FB43440070B5041C00253848436912219B0708D5364A1068364A106050304079122800D8011C43209EF76EFF324BA360324B2361201C0830ACF70FFE2168086063681D60ACF778FE201C1030ACF705FE216808600420ACF787FE6061062801DAACF76AFE201C0830ACF7F7FD216808606368002018600420ACF776FEE060201C1030ACF7EAFD216808606368002018600420ACF769FE6061E368C61A301CACF7B9FE042817DD01350C2D14D0301C042E08DDACF7AFFE8100081A2169081802382061CFE7ACF7A6FE8100081AA168081A0230A060C6E7A16820690B1AE3614018C30F18184310236270BDC046181B0800D4CC0800A0A40900FF03000001FCFFFC
:01443F00FF7D
:3031940000B5011C6831CB78002B07D04B7A002B04D18B78002B01D089F752FB00BDC0462CBE0500249C0900300308006D3109006D
:3C45740010B5A5F7D5FA0B494B699B070FD50A48036801200343084803600A249DF752FC013CFBD1044803685B085B00036010BC08BC1847181B0800F0FC0E0061
:FB445400F0B5444D2B68987B9DF73DFA46082B68996C301C9DF7D2F9041C2868011C94314A88002A10D094420ED9037D0B2B0BD00D2B09D072F7A1FA2B686433197F012000037CF773FF64E00B7D002B06D0CB88F31A1B041B0C9C4200D81C1CC36F6430002B06D00B89F31A1B041B0C9C4200D81C1C8A88B31A1A04120C944200D8141C0B881F1FBA4204D3CB7C022B01D30023CB74214E33889C4204D80020BA422ED303202CE073889C4201D8042228E0B3889C420BD9007F76F7C3FD002814D0037C112B11D115494B889C4203D829689431052215E08B889C420DD82968943106224A745E2383740CE0F3889C4203D829689431062204E029689431072E
:25454F002200E0021C4A740B7E012B04D1531F012B01D804234B74F0BDB421080034020800EC020800C4
:1845B00010B5094C2C220949201CC0F7E3F90849E160084B1C6010BD3C
:2445C800C27B4A4002D0838C05490B607047C046A4A4090034CC0500C945090010040800CC8A0E00C4
:D0461400F0B581B0041C00210091C56D8726F600002D04D1301C9CF7A8FF051E03D0301C9CF7A3FF0090264F3B68002B08D1301C08309CF79AFF3860311C0831C0F7BAFC20480368002B0DD1301C08309CF78DFF1C4A1060311C0831C0F7ACFC19480368002B07D03B68002B04D0002D02D00098002817D1E02300201851E565E4210B59DB0208D46358104803430B515022206807217FF7D8F90D480368002B0DD19CF770FF0AE0E5656060E4221359064883431351206807217FF7E7F9002001B0F0BD444408009C4408000000100060030800EC
:5C46EC0030B5E4221358012109058B431350051C7BF72CF90024002800D0EC65E86D002802D09CF75DFFEC656868002802D09CF757FF6C60074D2868002802D09CF750FF2C60054D2868002802D09CF749FF2C6030BDC046444408009C4408008E
:1847480000231360012805D10123DB040B6007239B0313607047000064
:70478800B0B503685B011948C21880270F404906490E9068002827D00568281C041C002F06D0437B8B4201D0002300E0012306E0037B5B088B4201D0002300E00123002B0FD0A84205D1137C002B02D1D37F022B0AD0111C08319DF7BEFC201C9CF7ACFE02E00068A842D9D1B0BDC0467C290800E7
:1A48140010B5002907D0041C72F79AF8201C70F705F8012000E0081C10BD18
:0A48440000B50B48B8F711FD00BDE8
:2E484E0030B5051C00240849A300C818C378AB4204D1A300C8180421C0F7AFFB0134082CF1D330BDC046B85208005047080067
:4C48840030B5104D0D24281C0022111C92F72EF9281C92F721F92035013CF4D130236343094818182C23195C022904D1406A002801D09CF789FE0134022CEFD392F7D6F830BDC0467C29080080590800FC
:FB49D000F0B584B0061C181C01AB07C300252C1C04F084FF00902F1C0199002918D0F37F022B15D1337C351C002B01D00C3500E008352A68101E00D01068002A07D01168914201D12C6001E00B6813600C6014E0357412E00A6801928A4201D1F76001E013680B6001990F60002C04D0236813602260141C01E0141C1260F1680029E9D115E01A680193111C9A4201D1B76004E0136801B40298036001BC0F60002C04D0236813602260141C01E0141C1260B368002BE6D1002D0BD02A68002A05D0136803602B681860286007E02860006004E0F37F022B01D10323F377009804F026FF12E02068051CA04201D1002401E0036823602F600399002904D0020B
:154ACB009900229EF73FFD01E09CF734FD002CEAD104B0F0BD5D
:019B04000A56
:2E49440010B5041C184908680007000F01280BD80B683F2000020340190A144A906EFFF7B5FF134A9378A37410BC08BC1847BF
:4A49720010B5041CB4F7C5FF0F498B78002B07D1A37C0B498878834202D0201CB5F795FD10BC08BC18470E020000049B0900A90300007102000000980E00A88B0E0038B0080074150800AC210800C2
:7448D000F0B582B0051C0E1C041CB0346946207B9CF7E1FF2C482D4A1178431AF6000198991940182A4B984201D3032005E00121284B984200D30221081C009943185808031D5808860176092188301C9CF778FF6788391C79F7F4F9381A4308AB80831958014009A0601422291C1B4804F0CEFF02B0F0BDF5
:0C4AE00000B592F743FF08BC1847000027
:4A4AEC0070B5C369DB021AD5061C041C9034E278002A16D1002914D181F761FE051CB66C002E0BD0A0880C214843124941431248C0F76EFB011C301CB8F789FCE570012000E0002070BC08BC184726
:424B360000B50B48072104F0E6FE0A48B8F78EFC0A4A1368002B00D00123002B01D076F79CF88B230648036000BD71020000D43000002C2D080020C50800EC2F0800EC8A0E0037
:144B800000B50121C90505480022B8F779FE08BC18470000C4
:144B94000248034948607047FC440800814B09009C45080012
:5C4BC00070B5041C0E1CEC300068002807D5E069C00104D5211C3C31201C96F715FDE06940021AD5656C07232B70FF236B70AE70211C2831E81C0622BFF7C4FE00236364E069012189058843E061EC210859400040080851281C95F761FF70BD3A
:164C1C00C169012292051143C161EC2319585A07114319507047D3
:164C3200C169032252051143C161EC2319585A07114319507047FB
:084CB40000F002F892F767FF1F
:3C4CBC0010B5041C8168002917D00868002814D0037B5B08132B10D1E37F022B0DD10A688A4202D10023A36001E013680B60002313609CF727FC0323E37710BD5E
:284D0C0010B50C1C0368002B0AD191F773FF002806D00121207F8140024803688B43036010BDC0467429080049
:184D440010B5041C04F0D0FDE369012189048B43E36104F0D1FD10BD15
:284D6C0030B5051C041CFC342068002804D0B8F772FB20689CF7DEFB281C85F796F82868FFF75FFD30BD000018
:0C4D940000B5FFF7E5F908BC1847000067
:744164001B480378002B18D01348C16BCB0714D581691022114381610521C26BD20708D503680822134303600368934303600139F3D1816910229143816170471001000024060800B805080038C8080034C808003CC80800CC05080070820E00FFFFF7FFFFFF0FFF45C80800FFFFFEFF98A4090030C8080092
:2E4DAC00124A1178880601D507200FE0C80601D506200BE08B0701D5052007E04B0701D5042003E00220CB0700D5032070477F
:224DDA000021064B1A78530700D504218175002141778177C177143001734173704754030800DE
:3C4E140010B50B4C2368002B06D10A489CF7ADFB20600849C0F7CEF8074C2368002B06D104489CF7A2FB20600249C0F7C3F810BD44440800400400009C440800BC
:165E380000B5102802D1FFF721FB03E0112801D1FFF78CFC00BD59
:784E5C0010B5021C00231370031C2833022018700123D370C878907306282AD80C1C01A1095C8F4406101A242E384200211C101C00F022F81FE0211C101C00F040F81AE0211C101C00F0C5F815E0211C101C00F0E9F810E0211C101C00F015FA0BE0211C101C00F06CFA06E0211C101C00F089FA01E01223137010BDED
:464ED400011C0831CA1D93079B0F02D10F23136005E00F231370002353709370D3700A1C0B3293079B0F02D10023136004E00023137053709370D3700123CB736B230B740B23C3707047AF
:FB4F1A00F0B584B0071C0C1C04260123029348790002097908430190B0F7B0FF00280ED06079000221790843B0F73DFF002801D102233B7000230293BE30027808E00198072179F73BFE002801D102233B7002683978081C5AD1BB4D2B7B03930123834001B40498034001BC0BD003B41C2141434B19DB8B0398834203BC05D10C21397005E0042E00D1061C01300428E3D300293CD1042E02D107233B7037E0281D0299002900D0281C012393400168194301601C20704340190199C1831030A3798374E379C374237A0A214B430382637A03750024002B02D0FF2B00D0012484760299417642750023191C1A1CC3760EC0038083720398002804D1A86010E7
:195015002101227EF71FFD0123B340287B184328730123FB7004B0F0BD0D
:52502E0070B5041C0125487900020E790643301CB0F72AFF002808D0301CB0F7BAFE002809D00025BE30017809E0301C072179F7BBFD002802D10223237000E001682378002B03D1281C00F06EFA20700123E37070BDF3
:C8508000F0B581B0071C0E1C0024C47308300090744D0123A3402868184002D00134082CF6D3082C01D107233B703B78002B47D1087A01282AD305D003280CD314D0042824D11AE02B1D1C206043C1180831301C00F03AF81BE02B1D1C206043C1180831301C00F086F812E02B1D1C206043C1180831301C00F090F809E02B1D1C206043C1180831301C00F0DFF800E012203870000615D131791C2060434019017173794371B1790A224A438271F379C371337A03720123A3402868184328600098C4710223FB7001B0F0BDF7
:AA514800F0B584B003910024251C0190221C0A300090261C3BE001352D062D0E3F490120A8400290E4235A58024001D0042DF2D3042D01D1072036E0601C0206120E0098035D9F1EE8316C016754031C60183F043F0C541C2106090E9B5C43704C1C2406240E009A535C8370111C3A1C61180330BFF7E4FBE4192406240E03990A680298024301352D062D0E01363606360E039802600198437A9E42C0D32048E430036813430360002004B0F0BDC9
:2651F20010B50C1C011C407A032801D8002801D1122007E0184A825C22700A31601CBFF7B8FB002010BDDD
:1A52C80030B5041C0D1C081C211C0A310622BFF755FB637AAB71002030BDCE
:B0521800F0B581B00F1C0090FF25002419E01D2040013058E040C0070DD5FF20813031182001401810220099093104F02BFB002804D13C7037E0FF2D00D1251C01342406240E044908E0C0464C9B09007C9C09007B990900059B09000878784E8442D6D3854222D2291C0098093001F018F9301C8030A900081800210160680081530720C00130180122AA40416A914311434162036A13430362FF2343557520C000335C013333543D70002000E0072001B0F0BD82
:B852E200F0B581B0071C0C791220082C01D3387006E00C200123A340574A11681940F6D03B78002B44D1534E0120A040326882433260311D1C20604345182B79032B1BD1002001238340134008D01C2343435B1801B4287A1B7A984201BC0BD001300828EFD304F0D2FA0090287A00F0EBFF009804F0D3FAFF232B722B79012B04D1E4363368A8688343336000253B480123AB400168194009D0031C44206843C018407FA04202D1281C00F01EFB0135082DECD30123FB7001B0F0BDD2
:44539A0070B50D792F4C4523DB00E2181378002D02D0002B12D001E0002B02D10C2303700CE00021231C083344264E43F6183C360023F370337101310829F3D315700123C37070BDF6
:8253DE00F0B581B0071C0E1C041C487900020D790543281C012179F7EFFB0090281CB0F7E0FC002363747079000231790843E073000A20740834009A002A05D0211C0931106878F7F3FD11E0281CB0F735FD00280AD0281CB0F7C5FC002805D0BE300078B3F70BFF607201E002233B700423FB7001B0F0BDC046E49D09007C9C090090A1090043
:2C5DD00070B5061C0C1C151C0821FF2094F7F3FE00280AD06B2383700123C37006714471210A8171C57194F771FE70BDC3
:3C5DFC00F0B581B0051C0091161C1F1C0D21FF2094F7DBFE041E0ED06B2383700223C3700571C6720773009905300622BEF7ACFD201C94F755FE01B0F0BD0000F8
:03997C00020410D2
:39997F00FB349B5F800000800010000000000000000000000000000000000000000000000000000000000000000000000000000000000000000000000076
:1C564C00012909D1436803208003034001208003834201D1012000E00020704797
:0C54600000B52021764804F051FA00BD90
:18546C0010B5754C2378002B03D0102100207EF70FFB0023237010BDB6
:D0548400F0B581B06D4E337B002B04D01021012200207EF7E0FAB0680130B060830701D1431CB36000210091012300998B40307B184046D0331C10331C204843C5182C1D0027AB7D002B14D0EA7DE989002000F07DFCAF75AF60AF810123EB76AB7E002B03D0207CB16843182B60A089B16843182360E37D002B17D0B0682B68984213D3A37D002B10D0217C0B182B60208900280AD06168BFF798FE0206120E6189002000F054FC67602781B3682068834208D3E37D002B05D0E775227D6189002000F045FC0098013000900428ADD301B0F0BDA4
:5C555400F0B581B000900C200022384D2C7B012393401E1C23401CD02B1C10331C275743FB185B7D8B4214D1B4432C732A1D0098002800D02A1C01238B40D94313680B401360002C03D1102100207EF77DFA002002E00132042AD8D301B0F0BDF7
:9C55B00070B5234C036DBE331D780123AB40616819403CD0002201239340217B194033D0231C10331C215143CE18311D737DAB422AD1737E002B27D1CB7D002B17D08B7D002B07D00B8901330B814B68124A82569B184B60104BC0560F228B56984204DD8889A26883180B6011E008750FE00A4BC0560E228B56984209DB8B7C002B06D101238B74C87402E00132042AC3D370BD4C9B0900589B090016010000B0
:1456E40000B58B21944804F00FF95A21934804F00BF900BD6E
:6C56F80030B5904D2B68002B03D0112100207EF7C9F900240123A340286818400FD02B1C083344206043C0183E23195C002906D0427D011C1731807D002300F063FB2B1C083344206043C0183C300023C37003710134082CDED32B607B4803604521C9006B1800211970E430016030BD90
:A8576400F0B5754F3B68002B04D01121012200207EF771F9786801307860830701D1431C7B6000250123AB403868184038D03B1C083344206843C418261C3C36B378002B16D078682368984212D37379002B0FD0217D0B182360A089002809D0A168BFF743FDE081281C00F03EF80023A360A381F378002B05D03379002B02D0281C00F032F87B68606883420AD3B378002B07D00023B370627D211C1731A07D00F0FCFA0135082DBED3F0BD3A
:3E580C0030B5C578AA1F1206120E44234B434A49CC1881780B071B0F4849C95C61771F2A00D90022A277062D05D94368991D201C1F30BFF7A1F83F340120207030BD52
:7C584A00F0B581B03B494522D2008A5C002A33D04422424308318D182F1C3C37FB78002B2AD0AA7F00920A321006000E011D3E2095F7A4F9041E1FD00220A0700120E070A61D687F2071A87D6071291C1731301C0622BFF772F8009A22730736291C1F31301CBFF76AF8EB8900997354201CB1F7C0FA0023FB703B7101B0F0BDE8
:FB58C600F0B584B00290039108274168C278130285781D43019553180322985600250090021C144E0123AB40306803400ED0331C083344246C43E4180E23E35E934202DA1A0612162F1C0135082DEAD3082D05D1082F03D2381C00F054F83D1C082D4DD244226A439419039961771C234B43054A0BE07F99090090A109007C9C090098A1090014E30500809C0900D218137823765378637693786383D378237708340022002B02D0FF2B00D00122271C3C377A713268002A05D172601121012200207EF769F87268237D9B182360638A9B1863600023BB70A360A3810099E18101990B069A0FA27502984168201C17300622BEF7E6FF0123AB4032681A433264
:0759C10060281C04B0F0BDDA
:4659C80030B5B54D44234343291C0831CC18211C3C310023CB700B71012282402B6893432B608B78002B06D0627D211C1731A07D002300F0FFF92B68002B03D1112100207EF748F830BDF0
:245A0E0030B50024051C00F008F9011E08D0281C00F008F8041C9F4A117A002900D10C1C201C30BD4F
:FB5A3200F0B584B0051C0C1C80786968019100236946CB704306D90F0391029100260123B3409249086818401ED0442070434718BB7F08370299994216D1391C17310198062203F012FF00280ED10121787D8140214009D06A460332311C281C00F05BF80121787D81408C430136082ED7D3002C4DD002990198FFF7D0FD002832D000270123BB400293234027D01C237B43794818180079032820D100260123B34073490868184016D0442070434018437F0830BB420FD1039A8275696817300622BEF748FF6A460332311C281C00F024F80298844302E00136082EDFD30137082FCFD3002C14D000270120B84020400CD0391C281CFFF7CFFE061C082E086F
:1B5B2D00D06A460332311C281C00F007F80137082FEBD36946C87804B0F0BDAB
:E05B4800F0B583B0071C01910C1C02924068FB78C3180320195600914F4E44236343301C0830C418251C3C35AB78002B21D011202356994203DD608A7368C31863606B79002B0BD0A3890133A381A368009A9B18A3600199381CFFF735FE3FE0237D002B3CD14049705C002838D002980121017034E010202356994224DB0121A970627D211C1731A07D012300F014F97068638A1B1863606B79002B02D0237D1B1823600023A381A3602F49705C002814D002980378002B0DD00199381CFFF703FE01232B7109E0237D002B06D12649705C002802D00298012101700099E18103B0F0BDC5
:FB5C2800F0B587B0C1780B0281781943069142680023FF2401A81CC01B4A1068002800D19DE04B06D90F04910198FFF7FBFC002805D001980022022100F0AEFB039000270198851D06988304990E8C1F0123BB4005930D4801680B407CD01C2179430E18317A0436012975D323D003295AD35CD004296FD15EE0C04690A10900B0A30900809C0900280200007C9C09002978002960D04B1CA3425DDC311C0831281C00F060F8002852DA2B78591C641A240624166D18012CEADC4DE0297800294AD04B1CA34247DC6978022926D3032904D9142902D0162920D116E000210DE0337A311C09312A18901C0222FFF7C6FC00282DD0009802300006010E00910803
:675D23001C29788B1E9842EBDB08E0337A311C0931A81C0222FFF7B2FC002819D02B78591C641A240624166D18012CC7DC14E0337A0398834210D10BE0B37B049898420BD1311C08310198062203F096FD002803D102980599084302900137082F00D271E7029807B0F0BD49
:465D8A00F0B5061C0F1C00240123A3403868184011D063010B481D187378687883420AD12A78B31CA878C118E81C03F072FD002801D1201C04E00134042CE5DB0021C843F0BD649D090094
:3856680070B5051C0E1C141C8B4214D9042B07D103782370437863700023E370A3700AE01022AB49201CBFF779F9321C291C201C0C30BFF773F970BDB6
:4456A000F0B581B0141C1D1CAC4215D0061C0F1C6A460232AC4206D22B1C211CFFF7D4FF2A1C391C06E0231C381C291CFFF7CCFF221C311C6846023004F0E0F80006001601B0F0BDA5
:D099B80031B80200815E0900695F0900E95F09004760090031B8020031B8020031B8020031B8020031B8020031B8020031B8020031B80200F960090031B8020031B8020031B8020031B8020031B8020031B8020031B8020031B8020031B8020031B8020031B8020031B8020031B8020031B8020031B8020031B8020031B8020031B8020031B8020031B8020031B8020031B8020031B8020031B8020031B8020031B8020031B8020031B8020031B8020031B8020031B8020031B8020031B8020031B8020031B8020031B8020031B8020031B802009E
:245E5C0030B5051CCC78342C00D30024A000AD4A8258281CC5F71EFD2823585D022800D1AC7330BDEE
:3A5E800010B50B1D9907890F01D11A6808E05B1AC9001C68CC402022511A5A688A402243A04B9A4202D8A0490A6001E0112303700123C37010BC08BC184759
:805F6800F0B583B0051C0C1C734A03CA01900291237D012B07D1A07EC0210140402902D112232B7028E0211C153101A80622BEF7F5FC6A46217D01A800F00EFA071C03F0A1FC061C624B1878874204D2391C201D00F07DFA0AE0009B834205D2227D01A9201D00F08DFA01E007232B70301C03F091FC281CFFF7BBFF03B0F0BC08BC184759
:5E5FE80070B582B0051C0C1C544A03CA0090019112232B704F4A137A002B19D0611D68460622BEF7BBFC21796846002200F0D4F9041C47490B7898420AD203F063FC061C201C00F07CF9301C03F064FC00232B70281CFFF78CFF02B070BC08BC18471C
:2060460030B5041C03F04FFC051C00F059F9281C03F051FC201CFFF77BFF30BC08BC184755
:6460F80010B5041C0A1C09790D480378994205D2D078FFF7ACFF2834002000E01220207010BC08BC1847C046B89909001F100400389B090090990900E44E080032150800059B090084A1090098990900A0990900A8990900B0990900E49D0900FF7FFFFFE9FC00003B
:5C5EBA0030B583B0051C0C1C9A4A03CA01900291B1F7E8FC002802D00C232B701CE095498B7D95490878834201D30723F5E7211D01A80622BEF749FD6A46E17801A800F08BF98D490B78984201D21723E5E7009AE17801A800F0B2F903B030BD14
:405F160030B582B0051C0C1CB1F7BEFC002801D00C2012E0211D68460622BEF728FDE1786846002200F06AF97D490B78984203D200F0B9F9002000E01220287002B030BD05
:9260660070B58EB00C1C364B06CB02910392354B06CB0091019205A98870CC70334DFF208130291820014118102204AE301C0830BEF775FCA1008031685802906000405B0390FF2001302918A0004058009061004031685A264908400190E92080002858E040C007C00F0AA9087002A9301C19300622BEF754FC6946301C1F300622BEF74EFCB31D1F221A48002194F7A0FF0EB070BDDB
:125F5600784A1178784B1A7A8B1AC3730223C3707047AD
:039B05002000003D
:10618C0000B5EB21A54803F0BBFBAFF7EEFE00BD5D
:2C619C0000B54121A24803F0B3FBA2480021C182017600F026F82022FF219F4803F078FB2022FF219D4803F073FB00BD4E
:3661C80000B5B2F725FB00239749CB750B7600F012F800200AE097490B5C022B05D301230B5420314318FF211970013092490B789842F0D300BD4E
:1461FE0000B5FF219048032203F051FBFF238E48437200BD12
:64621200F0B5061C0F1C151E01D0FF231360002422E08148011CC031095D002915D0FF2101310122A24041581140FA07D20FA240914210D1062161430818311C062203F024FB002807D1201C0BE0002D03D02B68FF2B00D12C600134754803789C42D8D3FF20F0BDFE
:4662760070B5061C141CCD076F4801230355031C20339918FF230B70EB0F9340016C19430164311C062353436348C0180622BEF76EFB6848037801330370221CE90F301C00F04AF970BD20
:4A62BC0010B55D4A115C634C2378994204D25B4BCB18FF2119701154594900230B540B1C20331A18FF231370012282400B6C93430B6406210B1C43434D48C018BEF766FE53480378013B037010BD2B
:2063060000B5EB21474803F0FEFA2022FF21474803F0C9FA2022FF21464803F0C4FA00BD37
:7663260070B53F4C0721C9016518295C420000231353221C803283009A1800231360221C403243009A180123DB031380DA11A3188200D2180023136001228240D6436B6A33406B62354A1378994203D2304BFF225A542A54FF2181316118000140181021BEF71FFE2B6A33402B627520C000235C013B235470BD70
:24639C0010B52C490A7890420AD20121814005E0224C236A0B4004D1490001309042F7D3FF2010BD8E
:F663C000F0B586B0041C01230193FF23181C03AD13C50120002A00D0136013490E1C049B022B08D3FF230133CD184036059B5B685F047F0C03E00D1C8035059B9F88002452E01D235B01CB1802931B68034041D0338801B40598022801BC1DD302B40D490B40019302BC26E0E49D0900689B0800E44E080066A4090064A10900289C080032150800FD4E080084A10900FA4E0800059B0900FF7FFFFF0093029B5B68E340DB07DB0F01B40598984201D0002000E00120029001BC019B002B11D0059B1B6801B42868834201BC0AD1009B9F4207D103940DE0002A03D01368FF2B00D1146040000435023601345C4B1B789C42A8D3039806B0F0BD4A
:3264B60030B50C1C594DFF2181316B182201011CD0181022BEF75BFA281C4030610008180121C9030180C8112818A4000021015130BD87
:6664E800F0B50E1C171C1C1C191CFFF7E0FF4A4D281C8030A1000818316801606000B18841531D2040012918FB07DB0FA3404A689A4313434B600123A3400A681A430A600B7A01330B72311C381CB2F703F90721C90169180855085D38490B78984201D2374B1C54F0BD38
:20654E0010B5141C0022FFF734FF30490B78984202D23249445400E0FF202F4B185510BD7D
:6C656E0070B5041C0D1C2E480368DB072DD50B78012B2AD16079C0210140402925D1201C00220221FFF715FF21490B7898421CD2204B820080329958221CA607B60F01D1116006E01170090A5170090A9170090AD1704100C95A2171090A6171E92189005958C140C807C00F287070BDA1
:1665DA00FF2807D0154A5076154A517215490B1802201870704784
:5065F00000B50C4A137898420ED2104A135C022B03D3021C002907D003E00A490A7E012B02D1111CFFF7E1FF00BDC046059B0900E49D09003215080066A4090064A10900389B0900E44E080084A10900289C0800EB
:16666C0010B54468B1F70AFC002803D1201C01D09AF760FF10BD33
:5266820030B582B00D1C141C0F210622224000D027216A46118090708304980ED07040209AF737FF0190002811D04022291C03F014F97FF7CAFB6D46E978019A8B18D870E878019943181C71281C79F7C8FA02B030BDA2
:7466D40070B5051C00244068B1F7AEFC00282FD1A14E7068002825D03168002907D00A68012001E0013012688A42FBD1011C9B48038899421CDA0C209AF702FF002817D06B684360EB784372AB7803723168002904D00B6803600860306001E030600060012405E0AA78E978686800F003F8041C201C70BD3D
:82674800F0B5051C0E1C171C88490868C0070BD50020FFF71FFE864CE075E07D85490B78984204D300202BE0814C0023E37501232360201D042103F0C5F8002001194319DB780B712B5C0B7501300328F6D3A5616677277703F0A6F8041C77488368002B06D176498160C060002383826DF7B0FE734874498160C060201C03F09BF80120F0BD6D
:6067CA0030B584B0041CB2F735FC002826D1644D686800281FD064480368E97EDB0703D508016849081802E0090167484018291C08316A46B2F7FFFA291C18316846032203F047F8002801D0002000E00120B1F7C0FB002802D00023A360E36004B030BDBC
:D4682A00F0B583B001244E4D50490B6800281CD1E87E0130DB070BD5FFF7ABFDE876E87E4C490B78984201D2002000E0012008E0E876E87E4E494B78984201D2002000E0012000283DD1041C41E0DB072AD5EB7EED69474EFF20013031189800421800922A1CA907890F01D1286808E06A1AC9001768CF402020411A50688840384300990860301C403059000918687900022A79104308800720C0013018C05C0121FFF792FE0EE00F2301AA13801835697AD1702B7A9370686802900B18181D1223037002E0122301A8038001A879F7B4F9201C03B0F0BD50
:3A68FE0010B5B2F715FD26490B689879012801D1AFF742FB21480378002B03D116480368DB0709D502F0E3FF041CB1F767FBB1F772FB201C02F0E3FF10BDB3
:6C69380010B512E00468211C844202D10023094800E02368036000230B606068002801D09AF7F2FD201C9AF7EFFD024908680028E8D110BDA08F080034150800389B0900A48F0800059B0900E89C080031CD0400A8B008004F7F0400649F09006E9C08006C9C0800E49D0900C04F0800F0
:6869B00030B500252C1C1CE07448011CC0310B5D002B15D0192D0ED2714A137E002B00D1147602230B55E0300555211C201C00F037F8013504E001230B55E030FF2101550134684803789C42DED3192D07D22C1C03E0201CB1F73AFF0134192CF9D36049CD75FFF7F4FB30BDF3
:386A180030B55F4B1C5C5F490B68DB0710D500215D4A13789C420BD25C4A63009D5A2B0405D463000121C90329439952012100E00021FFF7D1FD30BDCB
:546A500070B582B00C1C4D4DFF2101316958C140CA07D20F4C4B195C4C4E3368DB0710D54B4E337899420CD24B004A4E9E5B330407D401228B004848C35800930196694602E0062148434119E035605DB1F7C8FE02B070BDE1
:606AA40030B5151C0024012928D14368032189030B40012189038B4220D100220221FFF77DFC36490B78984216D2354A4300995A0B0404D543004904490C99520124002D08D03149405C2A4A1378984206D2211CFFF77CFD082002E0022000E0002030BD88
:486B040070B500242948255C294A507A2118204A1078BEF78DFB061CFF2D11D0FF280FD0011C281CFFF792FF2248835D4355B54206D0011C2039731801211970FF2383550134032CDED370BDB5
:746B4C0030B51048437EFF2B19D00024251CFFF7D3FF211C0BE0164A505C022806D301305054505CA04201D9041C0D1C0131064803789942EFD303490D76FFF73AFB30BD689B0800E44E08003215080066A40900389B0900059B0900249E0900E49E090064A10900FD4E080084A10900489C0800289C080092
:906BC00010B582B01D4C21684306D80F6B469A07920F01D1196006E01970090A5970090A9970090AD970164C216801AC2170090A61706946B1F7A2FD0006000EFF2819D00021104A535CFF2B11D15054193A127E0D4B5A720D4C0223235489181920BEF729FB0006000E01232354181C03E001310329E6D3002002B010BDC04680980E0084980E00FD4E080084A10900289C08005C
:A46CA200F0B5051C13235B049F4F3B60082105206EF774FF9D4F3B689D4803403B603B68C00703433B608B4F3B6802273B43894F3B60974C984820620123974F3B60974FB868606278686065A8692430C17880220A43934F3A60934E8378B07B002B0ED1924D0021B1F79DFCB169081C243042781302007B18430022B1F7AAFE09E00121B1F78FFC8A4D8A4A13680120400603431360884805608848838A8848036000232360F0BD99
:306D46000523838183692633187801280FD10021CB4382490B6000234B607D490B68802003430B607A490B68800403430B60704734
:566D760000B5C369002B23D013235B04694A13605F4A13685D4A13605B4A1368594A1360554A1368644A13607248724A11684160724A11684161714A11688160714A13680360704A1368704A136061486FF77DFE08BC184700003A
:6C6DCC0030B5052383816C4A116806220A40062A02D181692A3108E08B0702D481692C3103E04B0704D481692E310B8801330B8013235B0449490B605049CB69002B12D1524C2568C37B012B0CD1236880208343236002209AF7B5FF80231D43A06899040843A060256030BC08BC1847E1
:186E380013235B043A4803604148C369002B02D1434803680360704705
:106E500000B5002901D1FFF724FF08BC1847000046
:56709000F0B50C1C171CAEF76EFE061C201DB5F74DFF051E1ED0B18D0B051B0D012040031843210408432B1CA907890F01D1186006E01870000A5870000A9870000AD8703A06120E2104090C281D92F7C9FC281CB4F7B8FAF0BD94
:2A70E60030B50C1CFF233D3343430548C51802F0FAFBA2352C8002F0FEFB30BDC046F44E0800349D080038B00800D6
:C06FD000F0B581B0051C0C1C08790002C978084352D00020AEF706FFFF2801D109234CE0071CAEF7C0FE0023038121790902E27811438186C186051C84F709FC2E1CB03673885808E8806379252B0ED2394800900521BDF7D1FF6179C8084907490F01228A40009B195C11431954B07BFF233D334343314819180091281CB1F7BCF82F4885662521281CFDF73BFC307B0021B1F7F1FA0523AB80381CB1F73CF900999E3101200870381C002100F035F8A279E179381C00F005F801E012232B7001B0F0BDED
:A0714000F0B582B00D1C041C002D06D1CC23195C002902D000239E490B80022D03D0291CB3F76AFD10E0E37B012B05D1236B002B02D046231B5BA381FF200830205C012802D8201CB4F77CF9924A10680A38904A1080012D20D16946A07B9AF784FB8E4D287800280BD100988007800F07D003280FD1884A13680A3B0198984209D3874E777A337A73726FF746FA77720120287002E0201CB1F7F8FB02B0F0BC08BC18476C
:2872420070B52C2267496748BDF79BFB66486649086066494160664A674901611830664C674D674E74C070BD6D
:FB73280070B582B0051C041C8034E37A002B08D0036DBE3319780820AFF79EFF0023A376E3726378032B28D0A87B9AF7C2FA4008218C431A1E04360C618C00291DD08E421BD36078012806D1688CBDF76BFF062803D13E2002E0042803D008202B6DAF33187003236370281C6FF71DFB2B6DBE3319780520AFF770FF58E06068002808D00090002301936946A87B9AF7E4FB002363606378032B38D0FF201930285A864230D825E0FDCC0800E4B60800EC010800AB210800642C08006C21080078E40500F4A3090078150800FD72090001750900417109001971090085760900E1710900349D080009C108003C9B09004C9B0900A87B86F7DDFD002804D12888
:357423001CB4F717F8002802D0A349C8780CE06378002B07D1A14BA87B185C032802D29E49887801E09C494878A874281CB3F7F3FE02B070BDA5
:2C72FC0000B5017D032901D0042902D1B3F739FD09E0037D062B02D100F008F803E0092B01D1B3F75FFD08BC18470000E7
:6476840010B5041C11490B689B0711D5C37B012B07D1FF200630205C002802D1201C70F72CFA8123185D012802D1201CFFF7D5FF10BC08BC1847C04674150800E3C00800FDCC08001C800E00FFBFFFFFBC8B0E003C9B09008603080014010000ECB008001CCD08009E
:26765E0010B5021C803202235370036D598909015184041CB3F787FC236DBE3319780C20AFF7FFFD10BD5E
:4674BA0030B5051C041C9C34036DB8331968A0889AF7A8F9002815DB2B6DB8331968A0889AF799F92B6DB2331988884208D340180131C901BDF785FEE070E078802801D98023E37030BD9E
:6271E000F0B5041C056D81300078002814D1A07B9AF773FB47082E1CB8363168381C9AF70EFB00281ADD3168381C9AF701FBEB785B0098420ADB0EE0201C012170F737F9002803DB6E4A13689C4204D1B23529880439884202DB201CB3F7B9FFF0BC08BC1847EA
:5476E800F0B5061E20D00768002F1DD0407CAEF73EFB051C707C182141430C484418786891F7DDFF99F75EFF381C99F715FF00233360217A01312172217A05480278A88D91F712FF00232372F0BDC046F4B008007C150800D7
:8077440070B5051C0E1C041C8034A37F002B1ED0B1F7E3FA184A537C012B09D9E37E002B02D1A08BC10603D5311C281CB1F7A8FACD23585D00280AD0FF230533E818837D002B04D04378002B01D1012383700B490B681B070FD56378022B0CD1FF201630285C002807D0A0898004800E0023002800D10123237670BDECCC0800E02C080000
:FB77C400F0B5041C051C3A4806689835A8880712F306D90FE9707307D90F0307DA0F002F04D0344803685B0300D5111CFF231533E0184378002B03D1002901D0012343708A4216D0AB79002B15D1002F08D0D0231859C168C91BC16002D48368DB1983600122AA71201CB3F7FDFD201CB0F7F0FD01E0002383713307DA0FA8884307D90F8A4234D11C4F397C0A0702D5B304990E2DD1184A13689B0303D5B3079B0F032B25D004214840A880251C5035AE87B304980E1CD020221149BB68181D02F02CF8CC342078800712D50D490B68012080030340580B0BD02B68BE331878AEF769FAAF303D210170012028870023AB87F0BDA88B0E00E02C0800ECCC08BE
:0978BF000080980E00BC8B0E0045
:1878C80010B51F4C2068002805D08008800099F733FE0023236010BDB7
:3C78E000F0B5051CC668B469002C16D0B1F7A7FB002812D1154F3A1C211C1331E01CB1F77FFA381C00F00AF80023AB60EB60A008800099F715FE0023B361F0BD2E
:16791C0000B582B0262369460B800190081C78F799F902B000BDC6
:2279320000B54368002B04D010220448002193F778FB00BDC046E49C080086A409001720000083
:9C797000F0B583B00291FF233D3343432248C618356D01F0B3FF371C90372C1CB0348E239A5B02998A1A1204120C638853433A6FD21851014909019101F0A8FFF37B012B0ED16B8B5B000093288B4000019A101841014909181CBDF735FCA0800098E080281C83F724FFF37B002B0ED1E68870086883A188019899F713FFE288011C101CBDF720FC301A400828830298431E3B800123BB7203B0F0BD349D0800C4
:B47A1400F0B581B00090AEF7ACF9041C0027364E336BDB071FD5B4421DD0251C2C354223A97D9A5D914216D1291C1031301C3C30062201F029FF00280DD101F04DFF051CBE36307800F036F8281C01F04DFF3078B0F762FC03E0C03601370F2FD8DB0098B3F7B3FD251C0123EB852C35201C82F79BF800980021AFF79BFA1C4A13681021DB0603D5A971201CB4F727FC201CB2F7E5FDBE342178FF223D325143144BC9187F23FF2023300B54A623FF2017300B5401B0F0BDD9
:407AC80010B5FF233D3343430C48C418201C80304178012907D1418C608CBDF7B3FB062803D13E2002E0042903D00820236DAF33187010BD2890080040150800349D080088
:BE7B1000F0B5051C046D3C4803689D4201D1B1F7FBFA281CB1F737F92E1C8036308901380ED33081308904237370002808D1281C6EF745FFBE3421780520AFF799FB3DE0707800281FD1A87B99F7BFFE4008B034A16899F755FE01239B0698420CD267883B1859014909381CBDF740FB7843A168081840014009A060A068002373700223EB74A86117E0022815D1B37E002B12D0F37A002B0FD1F089318A431A1904090C164B994207D2002902D0281C00F007F8281CB3F78AFA281C6FF7A3F8F0BD85
:427BCE0010B5041C006DB2231A5A4A43A3699B1AA3617834238BE3820369DB04DB0E0A1C5A43E07825234B4325339B1AC018252176F787F8E07010BDC0466C210800FF7F000057
:8C7C4C00F0B5051C1F49FF230533C418E378980000230B544318581C00230370AF692B6D1889421C267C688C5043B04063681B1858014009381A01239B06984220D2B31D20789840A368D901EB7B002B00D15143E268824200D3101CBDF7AAFA011C802800D980219F352970074803789E4202D2701C207404E000230434191C381C0BC4F0BDC046ECB008006F150800DF
:8C7CE400F0B5061C071C9C373888102101401D490BD01D4BF518EB7898000A5C9301AA68D218AA604318597811E0174BF518EB7898004118487800280DD08C78097861438901BDF769FAA9680918A960211C8B01E868C018E8602B7C002B11D1E86800280ED0AB68D901F37B002B03D1336D1A8901325143BDF750FA802800D98020F870F0BDC046ECB008000401000040
:587D7000F0B50D1C114C20600B68DB0701D599F746FD0F4E0020706637680E48384030609AF752F89AF750F82868E0606868A060022070669AF748F89AF746F89AF744F837600020E060A060F0BDC04600820E001C800E00FFFFFFFD2B
:787DD00030B5041C80304378002B1BD10323E374252101230B55837E002B07D0236DD98B09014184A36903840123C372618CA06975F786FF238C984204D02084216DB03188800880FF230133E158E518A06999F7F7FC216DB2310A88011C101CBDF7E6F9011C201CB3F73AFAA3692B60201CB1F748F900236B7130BDFE
:FB7E5800F0B581B02F4806682F4805682F480378002B52D12E480368AB4203D12D480368B3424AD02C4C2D4FFE20284007D1002D03D02B480368DB0301D5002E1CD063681B071B0F022B02D002209AF74DF825480078606324480078A06368F7CBF901F031FD822141432068642250436430BDF799F9431C3B6018E063681B0702D000209AF732F800206063A063184A13680093174A1088392109014143181CBDF782F9386014490098BDF77DF9134908603868A06107490D6007490E6001B0F0BC08BC1847C04614CD0800B4C4080008C30800B8CA0800189B09000C000F00DC5E0800FC0A080009C308000AC30800C02D0800E80A080020CF01009C000FDD
:017F5300002D
:647F900030B5041C15490B685D78B2F753F9022C01D0042C16D1281C203083F79FF8042C07D10D4800231A1C191C93F73BF8022102E0022C03D10821281CAEF7FBFF281CADF778FF06490B689879012801D1ADF7DAFF30BD98B008000E200000C49C0800C89C08008E
:F8800000F0B5041C00216FF742FA002803DA01234E4843716FE0061C251C7835687A00280DD1A07B99F759FC4008236DB833196899F7F5FB002804DC687A002805D0002E03DD201CB3F7B3F855E0E37B012B03D1002801D101236B72A878802101433C4A1160082105206DF79AFD384A5379002B41D1B1F751F8374F381C052101F046FC03233B74201C00F037F8B1F702F8EB8A002B0AD1FF201630205C002805D1B1F73BF83B7C082003433B740023AB74FF230533E6180023F375201CB3F77EF9264A13780021002B00D101211170F078FF2806D16B7A022B03D1081CF070A3697360012805D8F1708B001C48C0187B7C8370201CB0F7A3F9F0BD6F
:7080F80030B5847C18490B788374051C012200216FF75FF8AC742C6DB223195B0239884200DB081C11494143E5208000BDF76AF8FF210531695C884200D3081C32342178490701D5012801D8002800D101200349487430BDA42C0800A4860E00ECCC08006C150800ECB008007415080071020000A4
:F884B800F0B50D1C041C002D17D171498B79002B0BD070490B69834207D16F4D2B68DB0603D546310120087063E0C17B807BB0F7ADF8201CB1F7D4FE5BE0FFF70CFF022D57D1664D2B1C5421085B0004271C52373988084358644833221C56329007800F01D1166808E0121AC0001168C1402026301A566886400E431E60A06B002835D157480368DB0716D5A06E4223195C3C300022FDF739FF53490B7898420BD243005149CA5A110406D4800050494058E8602A61802013E0A26ED06BE860161C3C36707900023179084328612B68802083432B60002042321178012900D180202B6803432B606868082108436860A06E806AE864F0BC08BC1847D4
:54830E0030B5041C002917D15F498B79002B0BD05E490B69834207D15D4D2B68DB0603D546310120087012E0C17B807BB0F783F9201CB1F7B2F80AE0022908D148308188027E53185A1CA28143885B1A438030BC08BC1847B6
:2086B000034B04480360044B044803607047C046889A090050150800B49A09006415080082
:2C9A88009F9504006D9904007F930400000000000F83090000000000F1810900000000000000000005990400C393040048
:2C9AB4009F9504006D99040091A2040000000000B984090000000000B185090093A304004549090073490900C393040098
:FB81F000F0B584B0A24F051C002601220092041CB1F72DFB4434207B01286DD305D0032809D33FD0042867D145E0E07D002834D006282FD131E0E07D002801D0062829D194480378002B0ED07DF708FE0121914A5156884207DA637E002B04D1281C6DF758FF267648E0237E002B45D0281C00F0A4F8061C637E002B3ED10423237386498B7986490B6000220092381CB1F728FCB86031E0431E012B2ED8281C00F08DF8061C29E0E07D002801D0062824D16388013B638020E0237E002B17D0E37D042B14D1A0884306D80F01900822744902A801F00CFBBB680198834207D102A9381C062201F0E3FA002800D10126281CB1F7BBFB281CB1F760F8002E050C
:2382EB00D03206120E6749A088AFF76FF80098002803D0281C0121B1F7A5F904B0F0BC08BC1847A1
:3286D00010B5041C6DF715FD201C6EF778F94A23002018536523195D0220AEF7C9FDA36EBC3318780021AFF7A5FF6C340220207010BD6E
:14872C0000B5011C32310B78FB2213400B70AFF7ADF900BD8D
:4C875000F0B5061C0F1C104D2C68A07B99F7BDF880084300991C608CA26983185801400999F74EF8041C002F0BD0B17B2B68987B6FF783F8002804D1032C01D8002400E0033C201CF0BDC0466C21080067
:2871180010B5041CC37B012B05D1AA480378002B01D101230370201CB3F7C1FD201CFFF7EBFF10BC08BC18477A
:6274580070B5041C0E1C994D2878002802D0013828702878012804D8954A136895490B401360002816D0201C9830C378002B02D18188CA060ED58379002B11D0311C201CB1F741FC2B78012B0AD9311C201CB1F70DFC05E0201CB1F7D2F8201CB3F77BFE70BDEF
:4883620030B54E4A11680B06D90F884218D14C4D2C68ADF7FAFDC1780B02817819430279130419434279130619438C4208D12A1F13681A0C41780B0200781843824201D0002000E0012030BDE3
:FB83AA00F0B583B0061C0024271C051C50352B7B002B5DD0012401A8B1F785FB00906B7B002B38D0EB7A012B09D14823985B0006C00FB0F7CEF8002801D1041C48E02E239B5D012B27D101A90098B0F7A2F92B4A1378984208D2EB7A022B1CD02B78022B19D1FEF704FB16E026480368002B00D041246408640023480378002B0BD00098012808D1029B03208003034001208003834200D102271C480368DB070FD52E20805D0022012800D10122009901A8FEF724FB071C082802D10120044308E0002F06D03A06120E074948363088AEF7AEFF201C03B0F0BDD0A4090068C30800002D0800108B0E0080980E00AC210800642C080008800E00A88B0E008884
:1384A500980E00321508007C9C09006C9C0800389B0900C2
:FB85B000F0B582B0041C071CB1F751F958373B79002B50D0FB78012B10D1251C2835AB79012B0BD17B79002B08D1287AFFF7C1FE002803D1201C6DF78CFD3CE0FB78012B39D8A56E6846B1F76BFA061C7B79002B10D16946281C3C300622BCF7BBF9291C42310E70281C3C30FDF7A9FF6C34012020702CE0251C2835AB79012B06D16946B0F784F8FF2801D0FEF7EEF916480368DB0710D5A8790022012800D10122311C6846FEF727FA022805D113494823185B0422AEF7B8FEA37C10498878834202D1201CB1F73FFF201C0121B0F7E9FF02B0F0BC08BC1847C046AC210800642C080008800E007C8B0E00389B0900059B0900249E0900E49E090080980E09
:0586AB00007415080039
:049AE000420500003B
:049AE4005E0400001C
:049AE8006204000014
:049AEC00420500002F
:049AF0006C04000002
:049AF40062190000F3
:049AFC006C040000F6
:049AF8004405000021
:049B000062190000E6
:FB87A400F0B587B0061C4568059581780A07120F0192C07803908A09009243191A79069200200490C84A13681879002804D1C7490B681B0600D4CAE10198062800D9CCE1C34C2378C3490879834202D3201CAEF745FBC0484188002923D00378002B10D06378002B04D0BC4899F730FC002818D000236370A370B74A508850214143B64805E02378B448002B04D15022514399F7D2FB06E099F71AFC002802D0201CAEF71DFB2078AB490B79984200D392E129231F1C47430297E11C8807800F01D10A6808E0091AC0000B68C3402022101A4A6882401A43029FA14B0199595CB954B818019F032F01D0052F5AD1984A13681B0600D446E100994170039FBB4D
:FB889F001F0372291C09300622BCF76CF80635E11C8807800F01D10B6808E0091AC0000A68C2402023181A4B6883401343029FF8180230291C0622BCF755F8019F052F17D10635E11C8807800F01D10B6808E0091AC0000A68C2402023181A4B68834013430299C8180F30039A0C3A291CBCF73AF8E11C8807800F01D10B6808E0091AC0000A68C2402023181A4B68834013430299C8182830F17872688918C978017001200490F0E00198042806D0684A1368F07871684018C078587264490868C379012B18D10099281CAEF7BDFD019A042A05D1AEF7DAFD002800D1D5E03CE0FF2803D10099281CAEF703FEAEF7E3FD002800D1C9E030E05B490B78002BBD
:FB899A002CD0019A042A18D1594F291C381C1030062200F076FF002800D0B7E0B87D03071B0F00998B4200D0B0E08023034000D1ACE04006400EB87510E00922835601200856834200DAA1E0291C49480622BBF7CCFF8023009803434548837501210491E11C8807800F01D10A6808E0091AC0000B68C3402022101A4A6882401A430299881800994170291C02300622BBF7ADFF33480378002B1CD0E11C8807800F01D10B6808E0091AC0000A68C2402023181A4B68834013430299C818F17872688918AEF7B3FE0006000EFF2802D0002104915CE006350398FA300006000E03900198E11C012812D18807800F01D10B6808E0091AC0000A68C24020231853
:F38A95001A4B68834013430299C8180021017215E08807800F01D10B6808E0091AC0000A68C2402023181A4B68834013430299C818039A0272291C0930BBF759FFE11C8807800F01D10B681BE0091AC0000A68C2402023181A11E0C04F0800E02C08005DC30800BC9C080093C3080014E3050068C30800B8AF0800C8AF08004B68834013430299C8182830F17872688918C97801700699480601D5002104910198022801D9062806D1301CFCF767FF0499002903D104900498002802D023780133237023780B490879834202D3201CAEF78EF90699080703D5301CAFF73EFA05E00598002802D0059898F7E1FC07B0F0BDC046BC9C08003B
:488B880010B5564C82209AF769FB000600160022A15600290ED0CB10CA1AC310D2187F23DB439A4201DA181C04E07F207F2A01DC10060016010609162170494A1368002B01D14848C17710BDB8
:B48BD00070B5002644480368002B01D185F7C8FE434C4449201C0F300522BBF7CBFE00252819C07B99F78EF836180135052DF7D33D48C36A5B011CD53C4803685B0518D400253B4803789E4213D001200A2D00D9022040194100374886F718FE002805D0291C201C0F3086F723FE013E0135252DE7D3211C0F313048052200F027FE002809D0211C0F312C480522BBF793FE63690120834363616369DB0707D4FFF780FA616901229143104001436161002070BC08BC184782
:268C840000B576F747FC00280BD11F480368002B07D114490B681D490868834201D1012000E0002000BD71
:80817000F0B583B0012100910027C0237B431A481C18206BC00729D5251CBC356B78002B24D1261CE38D2C36002B1FD0B379002B02D00021009119E0211C0C310F48052201F074FB002811D00223B371201CB4F720F801A9201CB4F708F801A9A878B3F7A2F8082201A9A878B4F724F901370F2FCBD3009803B0F0BD28900800004F0800F8
:128CAA0000B5B821194800F02CFE00230B4A137000BDF7
:608CBC0010B5041C15480368002B0BD0201C002186F7D8FD1821201C86F7D4FD4E21201C86F7D0FD10BDC046DCA40900B4C4080050370800F4460800F44E08005420080020040800A4030800E0340800004F080010CD0800E4C708009034080014CD080030
:FB750000F0B581B0041C061C88360027B780F774FF230533C518EB7D0133EB75C37B012B14D16B78002B1AD1694803689B0716D5A07B9AF7D2F980084100A06981420ED09AF766F940008421085108E001236B705A480378A3740123DB07AB61AF705C4800680090830723D5EB7D012B07D17EF76DFC011C201CAFF704FF01F005FB55484379022B14D1236DBE330068197888420ED17EF75BFC4F4B991D1A7988541879411C0720BDF766FE4A4B18714A4B1F707EF74CFCA874009906220A40062A2FD1A07B9AF78AF94008308344496258D00107D4012109061143404AA150201CFFF76CFF236DBE33187886F727FD201C00F0E9F8E878012804D839498092
:6375FB00000B5C01330B54E37B0099201C002B02D1FFF724FF01E000F097F8201CB1F71DF8B77014E0AF758B070AD5B0782E490B78984205D2E37B002B02D00130B07006E0337C002B00D03774201CB3F7B2FD0098830702D5201CFDF7ADFF01B0F0BC08BC18473C
:188D3C0000B576F7A9F9002805D11848437D002B01D177F7E8F900BD34
:188D540000B576F79DF9002805D11248437D002B01D177F7DCF900BD3A
:268D6C0070B5051C0E1C0024C02363430C481818036BDB0703D5321C291CB3F781F901340F2CF1D370BD00
:228D920000B5064877F7B8F97DF701FB13211620FFF7E3FF00BDE44E0800289008009C4508004B
:049B08000000000059
:089B0C00FFFFFFFFFFFF000057
:228DDC0070B5CD1C114C00F083FD061C291C201D0622BBF7C9FD301C00F082FD0123237070BDB7
:148DFE0010B5041C0E3009490622BBF7BCFD0623E37010BD10
:268E12000549002805D105480B78002B02D0081D00E003487047089B09000C9B090064000800B09C0800FE
:2871180010B5041CC37B012B05D1AA480378002B01D101230370201CB3F7C1FD201CFFF7EBFF10BC08BC18477A
:0871100000B5FDF713F800BD06
:28413C002449C37B002B04D1FF220632805C012806D108680002000A0122920602430A600B68174803607047A9
:287F680000B51E48037B022B0AD10C211C4800231A1C93F75BF80120000577F79BFE02E00420B0F784F900BD75
:848E580070B5041C08790002C9780843ACF7ACFF051C01D1122331E0006BC0051ED40026281C3030817810220A40296B09D0890502D50C23237012E0286B1149084328630DE00F4A1143402211432963C37810210B43C370281CAEF7F3FD00E00126A078000261780843217892F7DBF8002E03D0281C0021AEF73EF928340023237070BD00020000B2
:208EE40000B52C2250495148BBF74AFD4F48504B186050498161504941615049416200BDE7
:308F040010B5041C5030007800280ED12B231B5D201C012B07D16DF758FD4C22115B0120AEF7ACF901E0B1F73EF810BC08BC1847A7
:288F340010B5041C2030C37A012B0AD198F7C8FC616B98F77AFC002803DD201C0021B0F79BFE10BC08BC1847E4
:FB8F5C00F0B585B0051C01220292002200923649041C08682034E37A012B02D1334A117801E0324A5178A97406220240062A4AD12F4A16683207120F0192010704D5301CFDF710FE009002902A4F019805282BD1E37A012B28D83306D90F207B414023D1ACF7D6FF79680391B968049103A90231062200F065FC002816D10298002813D0281CB0F79EFF0099002902D0281C6DF78AF8281CB0F73EFEE07A012800D003204C22515BAEF73EF913490B681B060AD50198052801D0032805D1391C3004000C0122AEF7DAF905B0F0BC08BC1847C04620E4050020A40900581508005D8F0900058F0900358F0900BC8B0E005C150800A88B0E0080980E00E02C0831
:019057000018
:20912400002809D1104A1068104A1368984201D1012801D1002002E08800411AC81E704759
:349144000B4A1068C306990F01290BD14007400F052801D8002801D1002001E002490868024908607047C046901C08004CA4090004300E0002
:6A91900010B5A44C201C042100F0B8FB7F21C943A01D072200F082FBFF23236000239E4803709E4803709E4803709E4803709E4803709E4B9E4803600123DB029D48038080239D48037000239C4803709C4803709C480621BBF7F0FE14219B48BBF7ECFE14219A48BBF7E8FE10BDF6
:6C91FA0030B5041C98480368002B04D000230360282300201855944D00216962A96278F7C9FB92480368002B07D175F736FF002807D18F48437D002B03D1012091F7FFFB04E076F765FE2834042020700023894A137089480378012213430370FFF79BFF281C8A300621BBF7B2FE30BDB6
:7A926600F0B5061C051C081C08356C4C2368FF2B20D076490330062200F00DFB002819D16079022807D12068ACF772FDC38D012B10D1002711E001280FD1206875F70FFFC1690906C90E0839062903D2FF210931475C02E0122333700EE0A11DE81D0722BBF75DFB8021A01D072200F0ECFA00232371AF710823F370F0BD70
:8092E00030B50C1C5B4D0331281C0622BBF74AFB637A564803701422211C0A315648BBF741FB1422211C1E315448BBF73BFB002347480370434CFF232360281C0021ACF733FD002803D1281C0121ACF72DFD002806D0C38D012B12D1BE30007802210CE0281C75F7E7FB002809D0C2691206D20E083A062A03D2006801212060617130BDFC
:0E9360000B7935480370CB78304803707047A6
:0A947800381CF9F77BFC6BF77EF956
:3C2D740030B5051C7CF7A4F9041C281C8CF733FA8C49201C2830062206F086FD00280BD1894C2560012363717F21C943A01D072206F082FD00232371002030BDCE
:0A948200281CF9F794FC6BF797F92A
:382DB00010B5041C0120A040C143814803680B4003608BF767F97D480368A34203D1FF230360002343717B48037B002B03D0211C012002F0B7FB10BDEA
:FB936E00F0B5052630480378002B50D12A4C2768FF2F4CD02079811D0720BBF774FF05062D0E607902280CD1381CACF7EDFCC38D012B3CD1A31DEA560024012622490E7016E0012833D1381C75F785FEC1690906C90E0B1C083B062B29D2A31DEA56FF230933C45C0123174803700A2900D10326144800211D4B1B579A420DDA0278013202700278B24212D301700F4A1378002B0DD092F78BF90AE0154B1B5701709A4205DD06480378002B01D092F764F90120F0BC08BC18473C9B090002C108000FC10800840308008603080010C10800C05D00009C070800A007080099070800D8C20800ADC9080009C1080011C1080025C1080024C9080054200800DC95
:0F946900CC0800E44E0800EEC00800E00A08003E
:0C948C0081B000F003F874F7B8FB00009A
:FB949800F0B582B0061C01917CF7D4FC051C534C6379012B12D180202368805D83420DD1A02295552079001985712079411C0720BBF7D4FE20710023494A1370494F341C6434217F01238B403868184038D0002201239340387B18402FD03B1C10331C205043C3180093181D5B7D8B4225D1009B5B7E002B21D0C37D002B13D0837D002B05D003890133038143685B1943600F2283569D4204DD8289BB68D31803600FE005750DE00E2283569D4209DB837C002B06D101238374C57402E00132042AC7D3351C9F2028569F357CF723FC2870251CA37D0C35002B15D02368DB0508D4224803691B010ED5201C90F7FEFB002809D00023A3610123EB720023AB12
:7D959300726B72201C8EF723FC23685806000F01990A5C002A04D0164B185CA072431E0DE012490B69DB000BD512490A6811684B031B0F984204D18B025B0F013BB3810CE0012323722B68FF20013083432B600D2309490B70201C74F79FFB02B0F0BDC0463C9B0900860308004C9B0900542008009EBB05001C2B0800E8C00800ED
:18917800002E02D00020E05504E0E35D002B01D0013BE3557CF7F1FC96
:0C7F5400381CFFF788F902B0B2F7FAFB06
:4C726A0030B5041CBE342178FF233D334B4363495918FF2208328B18FF221A709F3140220A705F493C30062202F003FB00280CD15D4D23782B6002236B717F21C943A81D072202F0FEFA00232B7130BD84
:087F6000FFF7A9F9B2F707FCD5
:4672B60030B5041CBE342178FF233D334B4350481D18081C203083F70EFF281C6FF7BBFB86F7DDFE4D48217803688B4203D1FF230360002343714948037B002B02D00020FEF72DF930BD98
:FB750000F0B581B0041C061C88360027B780F774FF230533C518EB7D0133EB75C37B012B14D16B78002B1AD1694803689B0716D5A07B9AF7D2F980084100A06981420ED09AF766F940008421085108E001236B705A480378A3740123DB07AB61AF705C4800680090830723D5EB7D012B07D17EF76DFC011C201CAFF704FF01F005FB55484379022B14D1236DBE330068197888420ED17EF75BFC4F4B991D1A7988541879411C0720BDF766FE4A4B18714A4B1F707EF74CFCA874009906220A40062A2FD1A07B9AF78AF94008308344496258D00107D4012109061143404AA150201CFFF76CFF236DBE33187886F727FD201C00F0E9F8E878012804D839498092
:6375FB00000B5C01330B54E37B0099201C002B02D1FFF724FF01E000F097F8201CB1F71DF8B77014E0AF758B070AD5B0782E490B78984205D2E37B002B02D00130B07006E0337C002B00D03774201CB3F7B2FD0098830702D5201CFDF7ADFF01B0F0BC08BC18473C
:0E96380083780F2B02D1032311480360704783
:1896460000B50F480368002B05D0002303600F21181C7AF720FA00BD63
:2E965E0000B5094902060CD40868012807D102230B6018220F2100207AF7F0F903E0032801D1022000E0002000BD149B090093
:049B1400010000004C
:1896A800044A1088012149020140480A012250407047C046E8C40800A0
:1297200000B500F0E3F8002320490B7000F0E6F800BD25
:0A97420000B5012100F006F800BD9B
:0A974C0000B5002100F001F800BD97
:4697560030B50C1C144D15490B78012B1AD10178032901D0082915D18378002B12D100F0BAF8002C03D02B7801332B7008E0041C2878013803D3287002208CF7EBFF201C00F0B1F830BD1E
:1497A400014908787047C046DDA40900B85208005400080032
:1097320000B51E4B984202D1081C00F001F800BD92
:08979C0000B5FFF7D5FF00BD89
:2497C4000F2304480360044803600448036004480360704730300E0030340E0030380E000C200E004C
:7097F00030B5051C18480368052B02D19CF7D8FB10E000F073F8041CA0F722FC02280BD0281CA2F774FBA0F717FC002804D1201C00F06CF8012015E0201C00F067F8281CA2F765FB041CA0F735FEA0F750FE204007D00648037823430370012080028CF78CFF002030BDC046B0C808003BC3080057
:22987A0010B5B3F763FB041E04D103480449416097F784FE201C10BDC046145208006D98090034
:0E986C0000B510208CF77BFF08BC18470000E9
:04989C007847000009
:0C98A00000C09FE51CFF2FE1FC4005000C
:0498AC0078470000F9
:0C98B00000C09FE51CFF2FE1CC48050024
:0498BC0078470000E9
:0C98C00000C09FE51CFF2FE1E0510500F7
:0498CC0078470000D9
:0C98D00000C09FE51CFF2FE17410050094
:0498DC0078470000C9
:0C98E00000C09FE51CFF2FE160E80100C4
:0498EC0078470000B9
:0C98F00000C09FE51CFF2FE17CD70400A6
:0498FC0078470000A9
:0C99000000C09FE51CFF2FE190D7040081
:04990C007847000098
:0C99100000C09FE51CFF2FE1304F050058
:04991C007847000088
:0C99200000C09FE51CFF2FE1CC510500AA
:00000001FF
